:100000000C94A3000C94DB000C94DB000C94DB003C
:100010000C94DB000C94DB000C94DB000C94DB00F4
:100020000C94DB000C94DB000C94DB000C94DA11D4
:100030000C9489120C94680D0C94DB000C94DB007A
:100040000C94DB000C94DB000C94DB000C94F00DA2
:100050000C94DB000C94DB000C94DB000C94DB00B4
:100060000C94DB000C94DB000C94DB000C94DB00A4
:100070000C94DB00F6121D1315141D1315146913CF
:100080008C131514E313F213040005000600070097
:10009000080009001E037300690078006B0065000A
:1000A00079006B006500790062006F0061007200EA
:1000B00064000000180374006500630068006B00B2
:1000C0006500790073002E007500730000000403C2
:1000D000090409022200010100A0FA09040000013C
:1000E00003010100092111010001224000070581DF
:1000F0000308000112010002000000086B746B731A
:1001000001000102000105010906A101050719E02E
:1001100029E71500250195087501810295017508EB
:1001200081010507190029FF150026FF00950675B6
:1001300008810005081901290595057501910295A9
:100140000175039101C011241FBECFEFD2E0DEBFC5
:10015000CDBF04B603FE18C080917001909171016B
:10016000A0917201B09173018730904BA740B04BC2
:1001700059F4109270011092710110927201109254
:100180007301E0E0F8E1099511E0A0E0B1E0E2E6FA
:10019000F9E202C005900D92A031B107D9F721E034
:1001A000A0E1B1E001C01D92A037B207E1F70E94C3
:1001B000530A0C94AF140C94000008950C94DD00C5
:1001C0000C947801CF93DF933F98479A84B18F7551
:1001D00084B985B1806A85B98AB18D7A8AB98BB1C3
:1001E00082658BB9C9E1D1E01882A5E1B1E01C922A
:1001F000E7E1F1E01082198211961C921182DF91E1
:10020000CF910C94D90186B18095982F991F992789
:10021000991F83B18095881F8827881F880F892B95
:100220001D9902C094E001C090E0892B80931701D2
:1002300089B186FB882780F991E08927499902C016
:1002400092E001C090E0892B4C9902C094E001C07B
:1002500090E0892B8093180142E050E067E171E063
:1002600085E191E00E946014892B49F081E0809340
:1002700012010E94C90D9093140180931301809183
:1002800017018093150180911801809316018091C8
:100290001201882391F080911301909114010E9422
:1002A000E10D459750F080911501809319018091DF
:1002B000160180931A01109212010E94DB0181E065
:1002C0000895E82FF0E0E75EFE4F808108950895DD
:1002D0003C9A44983E9A4698269A2E98249A2C98AE
:1002E000559A5D98529A5A98539A5B980C94DE00EE
:1002F00080E00E946101873049F481E00E94610141
:10030000873021F40E94F3040C94160E089581E0C6
:10031000089581E008950C94890108950C948D014D
:100320001F93CF93DF9300D000D01F92CDB7DEB7DD
:1003300049835A836B8330911C0189819A813111E1
:1003400014C0662359F0222349F00E942806182F72
:10035000682F89819A810E94CC0503C00E94FB0509
:10036000182F69817A81812F04C00E942806698133
:100370007A810F900F900F900F900F90DF91CF9197
:100380001F910C942909FC01262F40815181628123
:10039000738184810C94900181E00895CF93DF9361
:1003A000EC0160E00E94C301BE01DF91CF910C948B
:1003B0008E010C9468010C94E00008950E94F304EF
:1003C0000E94DD012FEF84E39CE0215080409040AB
:1003D000E1F700C000000C94160E0F931F93CF930B
:1003E000DF93EC0161E00E94C3018C01BE010E9419
:1003F0008B01882349F1BE01C8010E944C0C88235F
:1004000019F1BE01C8010E94600A8823E9F0BE010B
:10041000C8010E94A80B8823B9F08A81882369F05B
:1004200001158CE5180731F00F3D1C4531F40E9491
:1004300092070AC00E94DE0107C0CE01DF91CF9172
:100440001F910F910C94870180E0DF91CF911F9154
:100450000F9108950E94490D0C9443020E94460298
:100460000C944F0D08950C94320281E008950C9481
:1004700035020895CF93C82F0E9433028C2F0E941B
:100480003702CF91089580E00C943A020E94A80CA4
:100490000C943A020E94A80C90911B01891721F03C
:1004A00080931B010C943A020895CF93882309F49A
:1004B00082C0C82F8238C1F40E94A80C81FD7BC085
:1004C00069E380910001909101010E94210D0E9439
:1004D00098062FEF81EE94E0215080409040E1F7A4
:1004E00000C0000069E319C08338F1F40E94A80C31
:1004F00080FD61C063E580910001909101010E943F
:10050000210D0E9498062FEF81EE94E0215080404B
:100510009040E1F700C0000063E5809100019091F8
:1005200001010E94230D44C08438C1F40E94A80C2C
:1005300082FD41C067E480910001909101010E9419
:10054000210D0E9498062FEF81EE94E0215080400B
:100550009040E1F700C0000067E4DFCF8CEF8C0F24
:10056000813AD0F46C2F80910001909101010E949A
:10057000EB0C882349F06C2F8091000190910101D0
:100580000E94230D0E9498066C2F8091000190918B
:1005900001010E94210D0CC080E28C0F883058F4BC
:1005A000C77081E001C0880FCA95EAF70E94CA06A9
:1005B000CF910C949806CF910895882309F45BC0DD
:1005C000682F823879F40E94A80C81FF54C069E337
:1005D00080910001909101010E94210D0E949806D6
:1005E00069E310C08338B1F40E94A80C80FF43C0B7
:1005F00063E580910001909101010E94210D0E940C
:10060000980663E580910001909101010E94230DFD
:100610000C949806843879F40E94A80C82FF2BC0B1
:1006200067E480910001909101010E94210D0E94D8
:10063000980667E4E7CF8CEF860F813A18F380E2E3
:10064000860F883048F4677081E001C0880F6A9592
:10065000EAF70E94D006DCCF8BE5860F833020F4CA
:1006600080E090E00C94BF0C685A673120F480E081
:1006700090E00C94D50C08951F93CF93DF93182F1F
:10068000EB010E945502209741F08FE99FE001970E
:10069000F1F700C000002197F6CF812FDF91CF91B5
:1006A0001F910C94DD02893319F060E070E002C004
:1006B00060E570E00C943C03882321F00E94CA0698
:1006C0000C9498060895882321F00E94D0060C947B
:1006D000980608950F931F93CF93DF93D62F172F6C
:1006E00012951F70FC0192811830E9F118F4123054
:1006F00028F0E0C0193009F4CBC0DCC0872F807F20
:100700007F70C72F882311F0C295C07F9923A9F06D
:10071000CC2379F080E28D0F883010F0D11104C025
:100720008C2F0E94CA0603C08C2F0E94DA060E94FA
:1007300098068D2F0E945502BDC08D2F0E94DD02AC
:10074000CC2309F4B7C080E28D0F883010F0D111AE
:1007500004C08C2F0E94D00603C08C2F0E94E0069C
:100760000E949806A7C0872F837009F045C0911199
:10077000A4C0462F429546954770440F440F862FDC
:100780008F7090E0A0E0B0E0042E04C0880F991FA5
:10079000AA1FBB1F0A94D2F764FF10C00FE010E03D
:1007A00020E030E004C0000F111F221F331F4A95C4
:1007B000D2F7009510952095309503C000E010E029
:1007C000980176957695472F4370BC01CD01602B3B
:1007D000712B822B932B423049F058F4413019F0A1
:1007E0000E941D056AC00E940B0567C00E942F056C
:1007F00064C00E94090561C0992319F0872F817098
:1008000001C08695882309F458C04D2F429546951E
:100810004770440F440F8D2F8F7090E0A0E0B0E040
:10082000042E04C0880F991FAA1FBB1F0A94D2F779
:10083000D4FF10C00FE010E020E030E004C0000F53
:10084000111F221F331F4A95D2F70095109520954E
:10085000309503C000E010E0980176957695472F1B
:100860004370BC01CD01602B712B822B932B423046
:1008700049F058F4413019F00E94A7051EC00E94AB
:1008800095051BC00E94B90518C00E94430515C0FC
:10089000C72FCF70992339F08C2F0E944F058D2FD1
:1008A0000E945C030AC0862F0E9463038C2F0E9463
:1008B000700503C01850123040F40E94A80CDF915C
:1008C000CF911F910F910C943A02DF91CF911F911C
:1008D0000F9108950F931F93CF93DF93EC016881DD
:1008E00079818A810E9475068C010E94CB050E9445
:1008F000F704B801CE010E946A03DF91CF911F91E6
:100900000F910895CF93DF93FC0190818181238122
:100910003481232B31F08F3F31F481E09F3F19F474
:1009200003C081E001C080E080FD0EC0EF01CF0177
:100930000E94ED01882341F0CE010E946A04CE019D
:10094000DF91CF910C94CE01DF91CF910895CF9399
:10095000DF93CDB7DEB72A970FB6F894DEBF0FBE90
:10096000CDBF4E835F83688779878A8761110E9434
:10097000E70685E0FE013696DE01119601900D92A4
:100980008A95E1F799818A812C813D81232B31F071
:100990008F3F31F481E09F3F19F403C081E001C033
:1009A00080E080FF05C0CE0101960E94820406C04F
:1009B000CE0101960E94CC018111F5CF2A960FB687
:1009C000F894DEBF0FBECDBFDF91CF9108950E9496
:1009D000E7060C94980680910001909101010E9415
:1009E000250D0C94E7040E94D7060C94EB0408959F
:1009F00008950C94F8040C94F9040E94FB0460938D
:100A000026017093270180932801909329010C946B
:100A1000E7040C94FD040F931F930091260110919D
:100A200027012091280130912901602B712B822B05
:100A3000932B1F910F910C94FD040F931F93009122
:100A4000260110912701209128013091290160236E
:100A50007123822393231F910F910C94FD040F9314
:100A60001F930091260110912701209128013091B8
:100A7000290160277127822793271F910F910C94DA
:100A8000FD040C94F8040E944105609322017093C8
:100A9000230180932401909325010C94E7040F9384
:100AA0001F9341E050E060E070E004C0440F551F28
:100AB000661F771F8A95D2F78091220190912301BA
:100AC000A0912401B09125018A019B01082B192BCB
:100AD0002A2B3B2BC901B8011F910F910C944305A0
:100AE0000F931F9341E050E060E070E004C0440FBA
:100AF000551F661F771F8A95D2F7409550956095D0
:100B000070958091220190912301A0912401B091D0
:100B100025018A019B01082319232A233B23C901AC
:100B2000B8011F910F910C9443050F931F930091EF
:100B30002201109123012091240130912501602B85
:100B4000712B822B932B1F910F910C9443050F93C4
:100B50001F930091220110912301209124013091D3
:100B6000250160237123822393231F910F910C94FD
:100B700043050F931F9300912201109123012091AF
:100B800024013091250160277127822793271F9127
:100B90000F910C9443050895362F292F220F920FA1
:100BA000890F982F9770A1E001C0AA0F9A95EAF7D4
:100BB00086958695869590E065E070E00E944914E0
:100BC000FC01E35EFE4F40E050E0632F70E0908157
:100BD0009B01042E02C0369527950A94E2F72170F6
:100BE000219529272A23292721934F5F5F4F4530DD
:100BF000510569F70895292F220F920F890FA82F09
:100C0000A77086958695869590E065E070E00E94D5
:100C10004914BC0140E050E080E0FB01E40FF51F07
:100C2000E35EFE4F208130E00A2E02C03695279504
:100C30000A94E2F721703327042E01C0220F0A9490
:100C4000EAF7822B4F5F5F4F4530510531F708952A
:100C5000BF92CF92DF92EF92FF920F931F93CF93A9
:100C6000DF938C01C0902201D0902301E0902401F9
:100C7000F09025018091260190912701A0912801F3
:100C8000B0912901C82AD92AEA2AFB2ACFE1D0E06B
:100C9000D701C6010C2E04C0B695A79597958795E8
:100CA0000A94D2F780FD04C0219790F7B12C07C0B9
:100CB000BC2EB8018C2F0E9444090197A9F38B2DFB
:100CC000DF91CF911F910F91FF90EF90DF90CF9028
:100CD000BF900895CF93DF93EC010E942806BE01D8
:100CE0000E944409DF91CF9108951F93CF93DF9322
:100CF000EB0190911C01992321F0CB010E946A061F
:100D000013C0882349F0CB010E942806182F682FB2
:100D1000CE010E94CC0504C0CB010E94FB05182F18
:100D2000BE01812F0E944409DF91CF911F91089548
:100D3000CF93DF93E0910001F091010180913B019D
:100D40008083E0910001F0910101908180913A014E
:100D5000892B8083C0910001D091010148E050E0CF
:100D60006AE271E0CE010E946014892B69F088E08C
:100D7000FE01AAE2B1E001900D928A95E1F7CE0161
:100D8000DF91CF910C94B40CDF91CF9108958091B5
:100D90003B01089590913B01892B80933B0108957D
:100DA000809590913B01892380933B010895109297
:100DB0003B01089590913A01892B80933A0108955F
:100DC000809590913A01892380933A010895109279
:100DD0003A01089580E090E00E94751421E0893E78
:100DE0009E4F09F020E0822F089582E090E00C945D
:100DF0006D1483E090E00C946D14CF9384E090E048
:100E00000E946D14C82F82E290E00E946D142C2F76
:100E100030E0A901582BCA01CF910895CF93C92F73
:100E2000682F84E090E00E947B146C2F82E290E0B7
:100E3000CF910C947B14AB01BC018FE090E00C943B
:100E40008D14AB01BC0183E190E00C948D1460E043
:100E500070E0CB010C94210760E070E0CB010E94B0
:100E60001B070C94270769EE7EEF80E090E00E945C
:100E7000991460E082E090E00E947B1460E083E0DF
:100E800090E00E947B14109226011092270110928C
:100E900028011092290160E084E090E00E947B1418
:100EA00060E082E290E00E947B1460E085E090E0E8
:100EB0000E947B1460E086E090E00E947B146FEF5C
:100EC00087E090E00E947B1440E050E0BA0188E0A7
:100ED00090E00E948D1460E08DE090E00E947B1411
:100EE00040E050E0BA0188E190E00E948D1460E09B
:100EF00087E190E00E947B1440E050E0BA018CE171
:100F000090E00E948D1460E070E080E290E00E942A
:100F1000991440E050E0BA0188E190E00E948D14FD
:100F20000C942C070C943307682F8EE090E00C94FF
:100F30007B140E94D50D609342017093430180930E
:100F400044019093450160933E0170933F0180936B
:100F5000400190934101089581E008950C94AC07FD
:100F600008950C94B0070C94B0070C94B3070C943C
:100F7000B0070C94B7070C94B00780E29AE00E9487
:100F80009E0C0E94BB070C94B9070E94B1070C94F9
:100F9000B0070E94230A0C9439020E94C00D0E94DF
:100FA000E2000E94C9070C94B5078F929F92AF92FE
:100FB000BF92CF92DF92EF92FF920F931F93CF9346
:100FC000DF93CDB7DEB72A970FB6F894DEBF0FBE1A
:100FD000CDBF0E940301982E81110E9499078CE3D6
:100FE000A82E81E0B82E00E010E0802E802F0E9415
:100FF0006101D82EF501C1905F01C826B1F40F5FE1
:101000001F4F0230110589F78FEF89838A831B8276
:101010000E94C90D8160782F9D838C8349815A81FC
:101020006B818D810E94A7042FC08091460181FDB4
:101030000E946701E12CFF24F3948C2D8F21F1F0A5
:101040000E94AE07882399F0EE828F82DF2081E034
:1010500009F480E088870E94C90D8160782F9A8703
:1010600089874E815F8168858A850E94A704F8017F
:10107000E45CFE4F8081F826F08206C0E394FF0C0A
:10108000F3E0EF12DACFBBCF81E0911001C080E036
:101090002A960FB6F894DEBF0FBECDBFDF91CF9179
:1010A0001F910F91FF90EF90DF90CF90BF90AF9086
:1010B0009F908F9008950E94D5070C944A02CF9379
:1010C000DF930E944909EC01811521E5920750F553
:1010D000811530E5930708F05CC0883E910580F4E7
:1010E000803E910508F0B1C08130910509F44EC0F1
:1010F00008F4A8C00497813A910508F4A6C0A2C0DC
:10110000811541E0940708F49DC08115904208F4D0
:101110009CC0C11580E4D80708F494C0DF70CE01EC
:10112000906A94C0811524E5920780F4811533E517
:10113000930708F069C0811542E5940708F04CC098
:10114000D82FCC27CE01816F906A80C08115984539
:1011500008F478C0C11589E5D80708F46DC0C11539
:101160002AE5D20708F06EC08C2F8F700E94DD092F
:1011700094E0D695C7959A95E1F7CF70D0E0DC2F33
:10118000CC27D0699E01282BC90160C081E090E086
:101190005DC074E0969587957A95E1F7282F2370C6
:1011A0003C2F337081E090E002C0880F991F3A9580
:1011B000E2F79C68AC01522B9C2F9F7096959695F8
:1011C000892F90E0EC01E5E0CC0FDD1FEA95E1F717
:1011D000CA018C2B9D2B3AC08370992721E030E007
:1011E00002C0220F331F8A95E2F79C2F96959695A1
:1011F000C92FD0E055E0CC0FDD1F5A95E1F7C22B87
:10120000D32BCE019C6822C08370992721E030E067
:1012100002C0220F331F8A95E2F79C2F9695969570
:10122000C92FD0E045E0CC0FDD1F4A95E1F7C22B76
:10123000D32BCE019A680AC0DC2FCC27CE01806F59
:10124000906A04C080E090E001C0CE01DF91CF91B0
:101250000895382F262F872F90E063E070E00E94DA
:101260004914FC01832F90E066E070E00E9449146D
:101270008E0F9F1FFC01E20FF11DEE0FFF1FE857BD
:10128000FF4F8591949108950E9429090E945F085B
:1012900008958238910569F1B0F48133910509F41C
:1012A0006DC048F48932910509F463C08A32910512
:1012B00009F469C008958533910509F455C089334F
:1012C0009105B9F00895833E910569F138F4803EA7
:1012D0009105B1F0823E910509F10895863E910590
:1012E000A9F1873E9105B9F1843E910509F064C0EA
:1012F00023C020915D0120FD4FC021FD4DC0089508
:1013000080915D0180FD44C080915E0180FF44C0FA
:1013100080915D0184FD42C083EE4DC080915D01EE
:1013200082FF38C0F5CF80915D0182FD33C080918E
:101330005E0180FD31C0ECCF80915E0181FF32C043
:1013400080915D0184FD2AC087EE35C080915D01EA
:1013500083FF26C0F5CF80915D0183FD21C0809180
:101360005E0181FD1FC0ECCF80915D0185FD1CC039
:101370001DC080915D0185FD19C016C080915D0181
:1013800086FD16C017C080915D0186FD13C010C098
:1013900089E311C082EE0FC080EE0DC080E00BC06B
:1013A00086EE09C084EE07C089E205C085E303C06C
:1013B0008AE201C081E390E0089590915D0192FF7F
:1013C0000DC0282F2871283019F4877F846006C04B
:1013D000282F2471243011F48B7F886093FF0DC077
:1013E000282F2871283119F4877E846106C0282FA0
:1013F0002471243111F48B7E886120915E0120FFDD
:101400000DC0382F3871383019F4877F816006C0DD
:10141000382F3171313011F48E7F886021FF0DC07B
:10142000282F2871283119F4877E816106C0282F62
:101430002171213111F48E7E886194FD877E08959B
:1014400080E0089508950E94EA06811102C00E947A
:1014500092070E94F506809346010E94FD06909334
:101460005E0180935D010E94220A0E94F906682FA6
:1014700070E080E090E00E94090560912201709187
:10148000230180912401909125010C9441050E9433
:10149000630F0E94CD070C946F0F0E94730F0E9480
:1014A0005B080C948D0F0E94670D0E944A0F0E94EA
:1014B000BD070E94470A0E944D0A0E94C507FBCF44
:1014C000CF93DF93EC01FB018281882309F43CC1B7
:1014D000C430FDE5DF0760F4CB3F9CE5D90788F415
:1014E0009E0122503C452431310508F02EC109C02F
:1014F000C236EDE5DE0729F0C63AFDE5DF0709F063
:1015000024C10E94FD0690935E0180935D01C1316C
:101510008CE5D80709F4C6C008F042C0C930ECE534
:10152000DE0709F49BC000F5C5308CE5D80709F447
:1015300085C078F4C330ECE5DE0709F478C008F024
:101540007AC0C230DC4509F0F5C080915D01816050
:10155000EFC0C7309CE5D90709F478C008F07AC01D
:1015600080915D018061E4C0CD30FCE5DF0709F4C6
:1015700087C058F4CB309CE5D90709F479C008F04E
:101580007BC080915D0188606FC0CF30FCE5DF07D4
:1015900009F480C008F082C080915D01877FC8C0D7
:1015A000CE3F9CE5D90709F471C000F5C531FCE5D3
:1015B000DF0709F485C068F4C3319CE5D90709F455
:1015C00075C008F095C00E94F30480915D018F778B
:1015D000AFC0CC3FFCE5DF07A9F108F054C0CB3F1A
:1015E000DC4509F0A7C080915E0140C0C230EDE546
:1015F000DE0709F489C058F4C1158DE5D80709F450
:101600005AC008F069C080915E0182602FC0C23666
:10161000EDE5DE0709F47CC0C63AFDE5DF0709F415
:1016200081C0C330DD4509F085C080E06EC0809187
:101630005D0182607DC080915D0116C080915D0179
:10164000886076C080915E0182604FC080915D01AC
:1016500080626EC080915D0180646AC00E94F30464
:1016600080915D01806864C0846062C081603DC01B
:1016700080915D018E7F5CC080915D018D7F58C03F
:1016800080915D0116C080915E0118C080915E015D
:101690008D7F2BC080915D018F7E4AC080915D015E
:1016A0008F7D46C080915D018F7B42C080915D013E
:1016B000877F8B7F3DC080915E018D7F8E7F15C0BF
:1016C00080915D0182FB222720F991E0922790FB17
:1016D00082F990FB83F92CC080915E01982F909540
:1016E00091708E7F892B90FB81F980935E0122C0DF
:1016F0000E94F30480915D0187FB222720F991E08D
:10170000922790FB87F914C081E00E94940712C0D1
:1017100080915D0184FB222720F991E0922790FBC4
:1017200084F906C080915D01982F909590FB80F917
:1017300080935D0180915D0190915E010E940E0792
:101740000E94F30480E001C081E0DF91CF91089511
:10175000CF93DF9386319C4541F5EB010E94C7068C
:10176000982F8A812091000130910101882379F01E
:101770009A7A81E009F480E080934701911102C0D8
:1017800069E201C065E3C9010E94210D0AC0809190
:101790004701811102C069E201C065E3C9010E94ED
:1017A000230D0E94980680E001C081E0DF91CF9177
:1017B00008950F931F93CF93DF93C42FD22FFC0173
:1017C00082818823C9F040934A010E94C90D9093F9
:1017D00049018093480180E28C0F883008F057C09F
:1017E000C77081E001C0880FCA95EAF7DF91CF91F9
:1017F0001F910F910C945C0380914A01481330C0F3
:1018000080914801909149010E94E10D883C910529
:1018100038F510E21D0FCD17B9F080E28C0F88303B
:1018200040F4C77081E001C0880FCA95EAF70E94B2
:101830006303183028F581E09D2F977001C0880F51
:101840009A95EAF70E945C03802F0E945303183098
:10185000F0F4D77081E001C0880FDA95EAF70AC08A
:1018600080E28C0F883098F4C77081E001C0880F47
:10187000CA95EAF7DF91CF911F910F910C94630302
:10188000802FDF91CF911F910F910C945303DF9123
:10189000CF911F910F9108950F939C01CB01243F8D
:1018A0004CE5340731F188F4293DFCE53F07D9F0D8
:1018B0002A3D4CE5340779F1283D3C45A9F506E27F
:1018C00021EE41EE68ED7CE52BC0263FFCE53F07AD
:1018D000E1F0A8F0273F3C4539F507E225EE46EE5A
:1018E00067EF7CE51DC007E225EE45EE69ED7CE57E
:1018F00017C006E221EE40EE64EF7CE511C007E27E
:1019000025EE44EE65EF7CE50BC006E221EE42EEEB
:1019100066EF7CE505C008E221E045EE6AED7CE576
:101920000E94D90B80E008C0FC018281882319F055
:1019300010924A0101C081E00F9108959093110126
:101940008093100108959093500180934F01089562
:10195000E0914F01F0915001309721F00190F0811A
:10196000E02D099480E00895E0914F01F09150013D
:10197000309721F00280F381E02D099408952091A1
:101980004D0130914E012817390771F090934E01A7
:1019900080934D01E0914F01F0915001309721F07B
:1019A0000680F781E02D0994089520914B01309134
:1019B0004C012817390771F090934C0180934B012B
:1019C000E0914F01F0915001309721F00084F185B2
:1019D000E02D09940895662349F0FC01329608969B
:1019E0002191621729F0E817F907D1F780E00895EF
:1019F00081E008959C01FC0132969FEF80E04191C7
:101A0000461789F09F3F19F4411101C0982F8F5F4D
:101A10008630A9F79F3F39F0F901E90FF11D97FDD5
:101A2000FA956283089508959C012A5F3F4FFC0157
:101A30004281461301C01282019682179307B9F7BB
:101A400008950C94FA0C0C94140D029626E0FC01F7
:101A500011922A95E9F7089508950C942C0D83E0CE
:101A6000809351010C942D0D811102C081E001C0C1
:101A700082E0809351010C942D0D0C94340D81E083
:101A8000809351010C942D0D0C943F0D08950C94EE
:101A9000460D0C94470D0C94460D0C94460D0C9479
:101AA000460D0E944D0D0E9403010E944B0D80E0E7
:101AB0000E946101811108C081E00E94610191E0F2
:101AC000811103C090E001C091E0892F089508952D
:101AD0001F920F920FB60F9211248F939F93AF9383
:101AE000BF9380915201811113C080915F01909149
:101AF0006001A0916101B09162014196A11DB11DEB
:101B000080935F0190936001A0936101B0936201A3
:101B1000BF91AF919F918F910F900FBE0F901F902B
:101B2000189580916701843031F10E942A02109249
:101B3000520120E488E190E00FB6F894A8958093D4
:101B400060000FBE2093600083B7817F846083BFF5
:101B500083B7816083BF7894889583B78E7F83BF76
:101B60000FB6F894A895809160008861809360001A
:101B7000109260000FBE08950E94F3040C942E0290
:101B800082E084BD93E095BD9AEF97BD80936E008F
:101B900008952FB7F89480915F0190916001A09112
:101BA0006101B09162012FBF08952FB7F894609141
:101BB0005F017091600180916101909162012FBF7E
:101BC00008959C014FB7F89480915F019091600156
:101BD000A0916101B09162014FBF821B930B0895E8
:101BE00078941F920F920FB60F9211248F939F93A8
:101BF000AF93BF9380915F0190916001A0916101CB
:101C0000B09162010196A11DB11D80935F01909377
:101C10006001A0936101B0936201BF91AF919F9168
:101C20008F910F900FBE0F901F90189581E08093B9
:101C3000E00080E28093D8001092C9008FE19EE41A
:101C40000197F1F700C0000087E090EBDC01809382
:101C5000700190937101A0937201B09373019CE0A5
:101C600088E10FB6F894A895809360000FBE90931A
:101C70006000FFCF80915B01089508950895CF9390
:101C8000DF9321E02093E9002FEF3091E80021500D
:101C900035FD06C035ED3A95F1F700002111F5CF7D
:101CA0002091E80025FF14C0EC0140E050E068E01E
:101CB00070E00E94EC0F8091E8008E778093E8003E
:101CC00088E0FE01A3E5B1E001900D928A95E1F76D
:101CD000DF91CF910895089508950C94440D60917B
:101CE000630181E0611101C080E00C942F0D90919F
:101CF000670181E0943009F080E0609163010C9409
:101D0000340D42E061EC81E00E94F0109091670197
:101D100081E0943009F080E0609163010C943D0D06
:101D200080916901833009F45DC030F4813071F035
:101D3000823009F496C008958A3009F482C08B304D
:101D400009F468C0893009F0A4C020C080916801FE
:101D5000813A09F09EC08091E800877F8093E80077
:101D600080916C0190916D01892B21F468E083E5ED
:101D700091E003C060E080E090E070E00E943710E6
:101D80008091E8008B778093E80008958091680146
:101D9000813209F07EC080916C0190916D01892B98
:101DA00009F077C08091E800877F8093E8008091F8
:101DB000E80082FD05C0809167018111F8CF69C0FC
:101DC0008091F200823031F48091F100813011F085
:101DD000863021F48091F10080935B018091E800CE
:101DE0008B7753C080916801813A09F052C080918D
:101DF0006C0190916D01892B09F04BC08091E80036
:101E0000877F8093E8008091E80080FFFCCF80917D
:101E10000E0136C0809168018132D9F580916C0144
:101E200090916D01892BA9F58091E800877F8093BF
:101E3000E8000E94251180916A0180930E010C94A4
:101E4000F30480916801813221F58091E800877F59
:101E50008093E8000E94251180916B0180935C01C2
:101E6000089580916801813AA1F48091E800877F0C
:101E70008093E8008091E80080FFFCCF80915C01B6
:101E80008093F1008091E8008E778093E8000C94B5
:101E90002511089584B7877F84BF0FB6F894A8955D
:101EA00080916000886180936000109260000FBE96
:101EB00090E080E80FB6F894809361009093610001
:101EC0000FBE0C943F0D0E9477110E94CA11E2EEE2
:101ED000F0E080818460808378940C942E1482E0FA
:101EE00091E00C94A30C809167018530A9F4809156
:101EF0006701853079F40E94910D809165018823F6
:101F0000B1F30E94510D882391F30E94D60F0E94D5
:101F1000F304EDCF0C94BC0D089508950C94900F2C
:101F2000292F332723303105C1F058F421303105F2
:101F300079F02230310591F582E290E022ED30E037
:101F400031C021323105E1F02232310501F126C0E4
:101F500082E190E024EF30E025C09927813091059F
:101F600049F028F00297D1F4E4E9F0E005C0EEEC86
:101F7000F0E002C0E4EBF0E0849190E09F0112C039
:101F8000672B61F489E090E024EE30E00BC0672B12
:101F900029F480E490E026E031E004C080E090E0A5
:101FA00020E030E0FA0131832083089584E089BD88
:101FB00086E089BD09B400FEFDCF8091D8008F7DF9
:101FC0008093D8008091E00082608093E00080914F
:101FD000E00081FDFCCF0895CF92DF92EF92FF9257
:101FE0000F931F93CF93DF93EC018B017A010E9433
:101FF0004411811133C0E114F10439F0F7018081FB
:102000009181081B190BC80FD91FC12CD12C0115A8
:10201000110519F18091E80085FD16C08091E80056
:102020008E778093E800E114F10449F0F701808194
:102030009181C80ED91ED182C08285E00FC00E9456
:102040004411882321F30AC089918093F100015043
:102050001109FFEFCF1ADF0ADACF80E0DF91CF91CD
:102060001F910F91FF90EF90DF90CF9008952091F6
:102070006E0130916F012617370748F06115710521
:1020800039F42091E8002E772093E80001C0B901CF
:10209000FC0120E06115710561F1809167018823E1
:1020A000D9F18530D9F18091E80083FD39C0809164
:1020B000E80082FD2BC08091E80080FFEBCF80918B
:1020C000F20090E06115710551F08830910538F407
:1020D00021912093F100615071090196F3CF21E025
:1020E000089709F020E08091E8008E778093E8005F
:1020F000D1CF2111D2CF0AC080916701882361F02E
:10210000853061F08091E80083FD0AC08091E8008D
:1021100082FFF2CF80E0089582E0089583E0089581
:1021200081E0089520916E0130916F0126173707E5
:1021300048F06115710539F42091E8002E7720935D
:10214000E80001C0B901FC0120E06115710579F1D9
:1021500080916701882309F43DC0853009F43CC0B3
:102160008091E80083FD3AC08091E80082FD2CC098
:102170008091E80080FFE9CF8091F20090E0611546
:10218000710559F08830910540F424912093F100B5
:102190003196615071090196F2CF21E0089709F05C
:1021A00020E08091E8008E778093E800CECF211167
:1021B000CFCF0AC080916701882361F0853061F03C
:1021C0008091E80083FD0AC08091E80082FFF2CF91
:1021D00080E0089582E0089583E0089581E0089505
:1021E000982F953068F59093E900981739F0709121
:1021F000EC002091ED005091F00003C0242F762FC9
:1022000050E021FD02C09F5FECCF3091EB003E7F9C
:102210003093EB003091ED003D7F3093ED00309135
:10222000EB0031603093EB007093EC002093ED00F5
:102230005093F0002091EE0027FDE5CF80E0089557
:102240008F708093E90081E008958091680187FF95
:1022500011C08091E80082FD05C080916701811165
:10226000F8CF11C08091E8008B770BC08091670197
:10227000882349F08091E80080FFF8CF8091E80042
:102280008E778093E80008952091E4003091E50076
:1022900095E64091EC00842F817040FF23C080912F
:1022A000E80080FD1DC080916701882399F085308A
:1022B00099F08091EB0085FD11C04091E4005091B0
:1022C000E5002417350729F3915011F09A01E1CF69
:1022D00084E0089582E0089583E0089581E0089500
:1022E00080E008954091E80042FFDDCF08950E940C
:1022F000D4110E94D711E0EEF0E0808181608083EC
:10230000E8EDF0E080818F77808319BCE3E6F0E0B0
:102310008081816080831092660108950E94D411AB
:102320000E94D7118091D8008F778093D800809138
:10233000D80080688093D8008091D8008F7D8093EA
:10234000D80084E089BD86E089BD09B400FEFDCFD8
:10235000109267011092630110926501109264015E
:1023600042E060E080E00E94F0108091E1008E7F0A
:102370008093E1008091E20081608093E20080918F
:10238000E20088608093E2008091E0008E7F80937D
:10239000E0000895E3E6F0E080818E7F808381E0B5
:1023A000809366010C948E111092E20008951092B1
:1023B000E10008951F920F920FB60F9211242F93F0
:1023C0003F934F935F936F937F938F939F93AF93BD
:1023D000BF93EF93FF938091E10082FF0BC0809148
:1023E000E20082FF07C08091E1008B7F8093E100D3
:1023F0000E942D148091E10080FF19C08091E200BD
:1024000080FF15C08091E2008E7F8093E200809172
:10241000E20080618093E2008091D8008062809326
:10242000D80019BC85E0809367010E946F0E8091EF
:10243000E10084FF30C08091E20084FF2CC084E082
:1024400089BD86E089BD09B400FEFDCF8091D8002A
:102450008F7D8093D8008091E1008F7E8093E10092
:102460008091E2008F7E8093E2008091E2008160A3
:102470008093E20080916301882311F084E007C01B
:102480008091E30087FD02C081E001C083E080937A
:1024900067010E94770E8091E10083FF29C080913F
:1024A000E20083FF25C08091E100877F8093E100F7
:1024B00082E080936701109263018091E1008E7F3A
:1024C0008093E1008091E2008E7F8093E200809112
:1024D000E20080618093E20042E060E080E00E94E0
:1024E000F0108091F00088608093F0000E946D0EE3
:1024F000FF91EF91BF91AF919F918F917F916F91DC
:102500005F914F913F912F910F900FBE0F901F90B1
:1025100018951F920F920FB60F9211242F933F938D
:102520004F935F936F937F938F939F93AF93BF93DB
:10253000CF93DF93EF93FF93C091E900CF70809129
:10254000EC00D82FD17080FDD0E81092E900809186
:10255000F000877F8093F00078940E94CD12109253
:10256000E9008091F00088608093F000CD2BCF705F
:10257000C093E900FF91EF91DF91CF91BF91AF91AF
:102580009F918F917F916F915F914F913F912F918B
:102590000F900FBE0F901F9018951F93CF93DF934E
:1025A000CDB7DEB7AA970FB6F894DEBF0FBECDBF8A
:1025B000E8E6F1E08091F100819321E0E037F20755
:1025C000C9F70E94900E8091E80083FF2EC1809190
:1025D000680190916901492F50E04A30510508F097
:1025E00024C1FA01E65CFF4F0C945A14803821F0A4
:1025F000823809F01AC108C0809164019091650188
:10260000992389F082600FC080916C018F708530B2
:1026100008F00BC18093E9008091EB0085FB8827CF
:1026200080F91092E9009091E800977F9093E8007C
:102630008093F1001092F100D1C0282F2D7F09F076
:10264000F4C0882319F0823061F0EFC080916A01F4
:10265000813009F0EAC0933009F080E08093650191
:102660002EC080916A0181112AC080916C018F7007
:102670002FEF280F243008F0D8C08093E900209174
:10268000EB0020FF1CC0933021F48091EB008062AE
:1026900014C09091EB0090619093EB0021E030E04A
:1026A000A90102C0440F551F8A95E2F74093EA0042
:1026B0001092EA008091EB0088608093EB0010920A
:1026C000E9008091E800877F8093E8000E9425114F
:1026D000ACC08111AAC010916A011F778091E300FC
:1026E0008078812B8093E3008091E800877F80933E
:1026F000E8000E9425118091E80080FFFCCF8091C6
:10270000E30080688093E300111102C082E001C001
:1027100083E08093670189C08058823008F085C0CB
:1027200080916A0190916B018C3D53E0950779F59A
:1027300083E08A838AE289834FB7F894DE01139697
:1027400020E03EE051E2E32FF0E050935700E491A7
:1027500020FF03C0E295EF703F5FEF708E2F90E097
:10276000EA3010F0C79601C0C0968D939D932F5FFD
:10277000243149F74FBF8091E800877F8093E800BC
:102780006AE270E0CE0101960E94371016C0609197
:102790006C0170916D01AE014F5F5F4F0E948E0F13
:1027A000BC01892B09F441C09091E800977F909378
:1027B000E80089819A810E9492108091E8008B77CD
:1027C0008093E80032C0803881F58091E800877FEF
:1027D0008093E800809163018093F1008091E8008C
:1027E0008E7772CF811121C080916A0190916B0127
:1027F00099270297D4F48091E800877F8093E800BE
:1028000080916A01809363010E9425118091630188
:10281000811106C08091E30087FD02C081E001C004
:1028200084E0809367010E94810E8091E80083FF1D
:102830000AC08091E800877F8093E8008091EB00D8
:1028400080628093EB00AA960FB6F894DEBF0FBEAD
:10285000CDBFDF91CF911F9108950895CF938091BF
:1028600067018823A1F0C091E900CF709091EC003E
:10287000892F817090FD80E8C82B1092E90080912B
:10288000E80083FD0E94CD12CF70C093E900CF9184
:1028900008950024552704C0080E591F880F991F5A
:1028A000009729F076956795B8F37105B9F7802DF3
:1028B000952F0895EE0FFF1F0590F491E02D0994D8
:1028C000FB01DC0104C08D910190801921F441507D
:1028D0005040C8F7881B990B0895F999FECF92BD17
:1028E00081BDF89A992780B50895A8E1B0E042E04B
:1028F00050E00C94A114262FF999FECF92BD81BD12
:10290000F89A019700B4021639F01FBA20BD0FB62D
:10291000F894FA9AF99A0FBE08950396272F0E9409
:102920007C140E947B14252F0E947C14242F0C946D
:102930007C140196272F0E947C140C947B14DC01DC
:10294000CB01FC01F999FECF06C0F2BDE1BDF89ABA
:10295000319600B40D9241505040B8F70895F89464
:02296000FFCFA7
:1029620032013A0E3F0E6B0E6C0E3D0E3E0E010012
:00000001FF
